:04000E0002080022C2
:013DFF00FBC8
:0300000002059462
:03000300021A03DB
:03000B00021A06D0
:03001300021A09C5
:03001B00021A0CBA
:03002300021A0FAF
:03002B00021A12A4
:03003300021A1599
:03003B00021A188E
:03004300021A1B83
:03004B00021A1E78
:03005300021A216D
:03005B00021A2462
:03006300021A2757
:03006B00021A2A4C
:03007300021A2D41
:10059400E4F5D9E5EF7480F5FF7402F5EF787FE4B4
:1005A400F6D8FD9000007F007E04E4F0A3DFFCDEBB
:0705B400FA7581210205190F
:05000600323237450015
:1006050075A4CF75D40875F2F875A5F875A71F758B
:10061500B0FF75A0FF7590FF7580FF75E10675E267
:02062500402271
:0A06A20075A14075F801E4F5A222ED
:0300160002064996
:0C069600E5A05401FFEF7002D322C32244
:10051900C207C208E4F5D91206051206A212069608
:1005290092073007371200167BFF7A00790612000E
:1005390076EF24FF92083008127D007C387F007E18
:10054900081205BB7F007E081201FAE4FFFE0FBF07
:0F05590000010EBE27F8BF10F5E4F5C002000E3A
:0906AC002321323030454655008F
:0B05680090005CEFF0FD90005BE0FFF6
:05057300900079EDF09D
:10057800120627EFC454F090007AF0900079E0FF5B
:0B05880012062790007AE02FF0E0FF41
:010593002245
:0B007600900067EBF0A3EAF0A3E9F0B4
:1000810090007174FFF0A37406F0A374ACF09000BB
:100091006E7401F0A37400F0A37408F090006A126A
:1000A10004E800000000E47F50FEFDFC90006AE0DF
:1000B100F8A3E0F9A3E0FAA3E0FBC31204C6504A97
:1000C10090006AA3A3A3E0FF7BA0E4FD12037E904E
:1000D100006EE0FBA3E475F0011204B0A9F0FAEFA1
:1000E10012049E90006AE0FCA3E0FDA3E0FEA3E001
:1000F100FFE4FAF9F8EF2401FFEA3EFEE93DFDE8ED
:100101003CFC90006A1204DC809C900071E0FBA32F
:10011100E0FAA3E0F9120458FF900008E06F706262
:10012100900001120471FF900009E06F705490007B
:1001310002120471FF90000AE06F704690000312F2
:100141000471FF90000BE06F70389000041204718D
:10015100FF90000CE06F702A900005120471FF906F
:10016100000DE0B5071C900006120471FF90000E0F
:10017100E0B5070E900007120471FF90000FE06FC9
:1001810060037F0022900067E0FBA3E0FAA3E0F99F
:10019100120458FF900019E06F702A9000011204B8
:1001A10071FF90001AE0B5071C900002120471FF64
:1001B10090001BE0B5070E900003120471FF900040
:1001C1001CE06F60037F0022900011E0900004F0BA
:1001D100900012E0FFA3E0900006CFF0A3EFF090B3
:1001E1000021E0900000F0900022E0FFA3E09000E9
:0801F10002CFF0A3EFF07F0143
:0101F90022E3
:1006490075B283E4F5A9538EF4758920758DF97512
:0B0659008BFFD28E75C15D43C1802273
:1005BB008F828E83D3E5829DE5839C5019758F03C3
:1005CB0075B7A575B7F1E4F0F58F2582F582740246
:0605DB003583F58380DE8C
:0105E10022F7
:0B037E00900074EFF0A3EDF0A3EBF093
:10038900C2052009FDD209C200D201D203D2047FDD
:1003990001C2C4C206D2C530C0FDE5C054F02480F4
:1003A900606224C0601A24E0600302043D90007674
:1003B900E0F5C2A200E43342C2C2C5E4A3F08076EC
:1003C90030C136300606D2C5C206806A30010CC279
:1003D90001D202900075E0F5C2805B300211C202C1
:1003E900900074E0F5C230034DD206D20080472058
:1003F9000044E4900077F0803D300404D2C5803693
:10040900D2058032EFFD900077E0FB3395E0FAC327
:10041900EB9D7480F86A98500CA3E5C2F0900077C0
:10042900E004F0D2C1900077E0B5070AC209C2C161
:10043900D2C48002D20530050853C0BF43C040C2B0
:0E04490009C2C03009030203A0900078E0FF52
:010457002282
:1005E20090005BEFF0900065E0FEA3E0FF12067D55
:0805F200900065EEF0A3EFF0AC
:0A05FA00EEFD900001E0FB12037E0D
:0106040022D3
:10066400900004E0FFA3E0C39F500D900001E0243C
:0906740002F0900005E004F02200
:10067D000FBF00010EC3900007E09F900006E09EA3
:09068D005006120664E4FEFF228F
:0801FA00900058EEF0A3EFF0B5
:10020200E490005BF0A3F0900061F0A3F090006531
:10021200F0A3F0900002E0FFA3E0900065CFF0A30E
:10022200EFF0900000E0A3F0E490005CF090005B3F
:10023200F090000504F0E4900060F090005BE06450
:100242003A6025900065E0FEA3E0FF1205FA9000F7
:100252005BEFF0900065E0FEA3E0FF12067D9000E8
:1002620065EEF0A3EFF080D3900062E004F0700638
:10027200900061E004F0900065E0FEA3E0FF12054B
:10028200FA1205E212056890005EEFF0900060122B
:1002920005E61205E2120568900063E4F0A3EFF0B0
:1002A200900063A3E0FFFD900060E02DF0EF90006E
:1002B20063F0A3E4F0A31205EA1205E212056890C6
:1002C2000063E0FEA3E04FFF900063EEF0FEA3EFB9
:1002D200F0AC068C08F509900060E02F1205E612DA
:1002E20005E212056890005DEFF0900060E02FF0EB
:1002F200EF706990005AF090005EE0FF90005AE0C3
:10030200C39F50581205E71205E212056890005F7C
:10031200EFF0A3E02FF0A3E0B4010AA3E0B4DA0502
:10032200E490005BF0D3900059E09509900058E00A
:100332009508501F758F0175B7A575B7F190005FCD
:10034200E0850982850883F0E4F58F0509E50970E7
:1003520002050890005AE004F00202F91205E712C1
:1003620005E212056890005FEFF0A3E02F700C9099
:0B037200005DE064016003020238221D
:01037D00225D
:10045800BB010689828A83E0225002E722BBFE02A2
:09046800E32289828A83E49322D5
:10047100BB010CE58229F582E5833AF583E0225040
:1004810006E92582F8E622BBFE06E92582F8E2228A
:0D049100E58229F582E5833AF583E49322A4
:10049E00BB010689828A83F0225002F722BBFE013D
:0204AE00F32237
:1004B000A3F8E0C5F025F0F0E582158270021583FF
:0604C000E0C838F0E8225C
:1004C600EB9FF5F0EA9E42F0E99D42F0EC6480C8AD
:0604D60064809845F0224D
:0C04DC00ECF0A3EDF0A3EEF0A3EFF02293
:1004E800A8828583F0D083D0821204FF1204FF1201
:1004F80004FF1204FFE473E493A3C583C5F0C58326
:10050800C8C582C8F0A3C583C5F0C583C8C582C85D
:0105180022C0
:10062700EF7E0024D0B40A00401624F9B40A004033
:100637000CB41000400A24E0B41000400374FFFE1D
:02064700FF2290
:00000001FF
